:10000000DB2801308F00AF308C00AF308D008D0BBE
:1000100007288C0B05288F0B032808000F3092004F
:10002000AF309000AF309100910B1428900B122844
:10003000920B10280800051401200510012008006B
:1000400005140120012001200510012008001B20BB
:100050002020080020201B201B201B20080020201F
:100060001B2020201B20080020201B201B20080014
:100070001B2008001B201B2020201B200800202004
:1000800020201B2008001B201B201B201B200800F9
:100090001B201B2008001B202020202020200800DF
:1000A00020201B20202008001B2020201B201B209C
:1000B000080020202020080020201B2008002020ED
:1000C0002020202008001B20202020201B200800AA
:1000D000202020201B20202008001B2020201B2067
:1000E00008001B201B201B200800202008001B20CC
:1000F0001B20202008001B201B201B202020080084
:100100001B202020202008001B201B201B2020203B
:10011000080020201B202020202008002020202054
:100120001B201B2008001B201B201B201B201B202A
:1001300008001B20202020202020202008001B2039
:100140001B2020202020202008001B201B201B20FB
:100150002020202008001B201B201B201B202020EB
:1001600008002020202020202020202008002020FF
:100170001B201B201B201B200800202020201B20D0
:100180001B201B2008002020202020201B201B20BB
:10019000080020202020202020201B2008002020D4
:1001A0001B201B2020201B200800012001200120F3
:1001B000012001200800FF308316860083120030E2
:1001C0008316850083128501061CEB20861C0C21FA
:1001D000061D861DE4287520382071207520D52045
:1001E0007520382071207520D52075203820712089
:1001F0007520D52034203820D5203F20C3206D2005
:1002000027205F20D52048205F20C9209F2027205D
:100210005420D5200E20080075203820712075202C
:10022000D5207520382071207520D52075203820E4
:1002300071207520D52034203820D5203F209320F0
:100240005C205C203A20CF202720D52048205F204A
:10025000C9209F2027205020D5200E200800000014
:0602600008000000080088
:02400E00F13F80
:00000001FF
